:100000000C945F040C94A3040C94A3040C94A30418
:100010000C94A3040C94A3040C94A3040C94A304C4
:100020000C94A3040C94A3040C94C40D0C94960E8D
:100030000C94A3040C94A3040C94A3040C94A304A4
:100040000C94A3040C9441230C94A3040C94A304D7
:100050000C94A3040C94E31C0C94A3040C94A3042C
:100060000C94A3040C94A3040C94A3040C94A30474
:100070000C94A3040C94A3040C94A3040C94A30464
:100080000C94A3040C94A3040C94A3040C94A30454
:100090000C94A3040C94A3040C94A3040C94A30444
:1000A0000C94A3040C94A3040C94A304FB0E1D0F46
:1000B00008101D0F08105F0F820F0810D70FEA0FEE
:1000C000DE12DE120C130C134E138A138A158A15D6
:1000D000A2138A159914991464158A158A1578152E
:1000E000000000810889248935812B850252E100B6
:1000F000E00000001E00140004001D0000774E0008
:100100001F001A0016001B00007F4C002000080092
:1001100007000600E2002A0021001500090019006E
:10012000E3004B00220017000A00050000004A000F
:1001300029002F0000002B0200004D002D00300090
:1001400000002B000000500023001C000B001100D9
:1001500000004F00240018000D001000E7005200BE
:1001600025000C000E003600E6002C0026001200D0
:100170000F003700007F28002700130033003800ED
:10018000007751002E8131853482E500E4000000C3
:100190000100C300C2003900010000002900010075
:1001A0000100010001000100010001000100010047
:1001B0000100010001000100010001000100010037
:1001C0000100010001000100010001000100010027
:1001D0000100010000000100010001000000010019
:1001E000000001000100010000000100000001000A
:1001F00001000100010001000000010001000100F8
:1002000001000100010001000100010001000100E6
:1002100001000100010001000100010001000100D6
:100220002A00010001000100010001000100C300DB
:10023000C200390001000000C20005520252E10074
:10024000010000003A001E022002220201005100BB
:100250003B001F0221022302010028003C002F0264
:1002600026022F0001002C003D0030022702300042
:10027000010052003E00240235003502000050000B
:100280000100360200002B0000004F000100370281
:1002900000002B0200004A003F003102380031000C
:1002A00000004D004000240021001E0027004B00EC
:1002B0004100250022001F0037004C0042002600AC
:1002C000230020002E002A004300380025022D00C4
:1002D0002E024E00C20005520252E5002800000026
:1002E000045205520852E100010000003A001E02CB
:1002F00020022202010051003B001F0221022302C2
:10030000010028003C002F0226022F0001002C00D3
:100310003D00300227023000010052003E0024025E
:1003200035003502000050000100360200002B00AD
:1003300000004F000100370200002B0200004A00BD
:100340003F0031023800310000004D004000240021
:1003500021001E0027004B004100250022001F0045
:1003600037004C0042002600230020002E002A0007
:100370004300380025022D002E024E000452055283
:100380000852E5002800000001000654C1003900B1
:10039000010000002900010001000100010001002E
:1003A0000100010001000100010001000100010045
:1003B0000100010001000100010001000100010035
:1003C0000100010001000100010001000000010026
:1003D0000100010000000100000001000100010017
:1003E0000000010000000100010001000100010007
:1003F00000000100010001000100010001000100F6
:1004000001000100010001000100010001000100E4
:1004100001000100010001002A00010001000100AB
:100420000100010001000654C10039000100000074
:10043000C30005520252E100A8000000440066001B
:10044000A6000000AA00B50045000000F200000070
:10045000A90000006800F000F100F100F400B6000F
:1004600069000000F3000000F500B4006A0000001D
:10047000000000000000B8000000F9000000FA00D1
:100480000000B9000000F9000000FA000000AC0014
:100490006B004600530000000000AB006C004A00F7
:1004A00050004D004900A9006D005200510051005C
:1004B0004C00AE006E004B004F004E000000AD003F
:1004C0006F00B100B30000000000AA00C300055295
:1004D0000252E50000000000075208520000E1004F
:1004E000A800000044006600A6000000AA00B500B5
:1004F00045000000F2000000A90000006800F000C4
:10050000F100F100F400B60069000000F300000003
:10051000F500B4006A000000000000000000B80010
:100520000000F9000000FA000000B9000000F90026
:100530000000FA000000AC006B0046005300000011
:100540000000AB006C004A0050004D004900A900BB
:100550006D005200510051004C00AE006E004B0087
:100560004F004E000000AD006F00B100B30000006E
:100570000000AA00075208520000E5000000000039
:100580000100C10001003900010000002900010044
:100590000100010001000100010001000100010053
:1005A0000100010001000100010001000100010043
:1005B0000100010001000100010001000100010033
:1005C0000100010000000100010001000000010025
:1005D0000000010001000100000001000000010016
:1005E0000100010001000100000001000100010004
:1005F00001000100010001000100010001000100F3
:1006000001000100010001000100010001000100E2
:100610002A00010001000100010001000100C100E9
:100620000100390001000000C100010001000100CB
:10063000010000002900010001000100010001008B
:1006400001000100010001000100010001000100A2
:100650000100010001000100010001000100010092
:100660000100010001000100010001000000010083
:100670000100010000000100000001000100010074
:100680000000010000000100010001000100010064
:100690000000010001000100010001000100010053
:1006A0000100010001000100010001000100010042
:1006B0000100010001000100010001000100010032
:1006C00001000100C1000100010001000100000063
:1006D00016034500720067006F0044006F00780049
:1006E000200045005A000000160345007200670014
:1006F0006F0044006F007800200045005A000000A1
:100700000403090409026D00040100A0FA090400B1
:10071000000103010100092111010001223F00072E
:1007200005810308000A0904010001030102000910
:100730002111010001224D000705820308000A096A
:10074000040200010300000009211101000122360A
:10075000000705830308000A0904030001030000E1
:10076000000921110100012239000705840310004E
:10077000011201100100000008EDFE071301000145
:1007800002000105010906A101050719E029E71585
:1007900000250195087501810205081901290595B3
:1007A000057501910295017503910105071900294D
:1007B0007715002501957875018102C00501098032
:1007C000A101850216010026B7001A01002AB70010
:1007D000751095018100C0050C0901A10185031662
:1007E0000100269C021A01002A9C027510950181C5
:1007F00000C005010902A1010901A10005091901B3
:1008000029051500250195057501810295017503DE
:1008100081010501093009311581257F950275088F
:10082000810609381581257F950175088106050C1B
:100830000A38021581257F950175088106C0C0051B
:10084000010906A101050719E029E7150025019511
:1008500008750181029501750881010508190129B2
:10086000059505750191029501750391010507191B
:100870000029FF150025FF950675088100C00000BE
:10088000000000000000000000010204060A0F172B
:10089000202C3A4A5D71879DB3C7DAE9F5FCFFFC6D
:1008A000F5E9DAC7B39D87715D4A3A2C20170F0A24
:1008B00006040201000000000000000000001124F6
:1008C0001FBECFEFDAE0DEBFCDBF04B603FE24C00B
:1008D0008091EF019091F001A091F101B091F201AE
:1008E0008730904BA740B04BB9F41092EF011092B3
:1008F000F0011092F1011092F20114BE84B7877FCB
:1009000084BF88E10FB6F894809360001092600075
:100910000FBEE0E0FFE3099511E0A0E0B1E0E6E002
:10092000FAE402C005900D92A433B107D9F721E093
:10093000A4E3B1E001C01D92AF3EB207E1F70E940F
:100940000A0B0C9401250C94000061110BC0FC01F2
:100950008281882321F085EE0E946B1103C085EE11
:100960000E94331280E090E008950895CF93609143
:10097000B1017091B2018091B3019091B4010E94D4
:100980000F1CC82FE0910E01F0910F01808182723F
:1009900019F0259A2D9A06C00E94431081FDF9CFC7
:1009A00025982D98C130B9F0C430A9F089EF8C0F8B
:1009B000823088F08EEF8C0F823018F4269A2E9AAF
:1009C00002C026982E98C550C23018F4279A2F9A44
:1009D00002C027982F98CF9108950C94B60456988A
:1009E0005E9825982D9826982E9827982F988FEF07
:1009F00090E0909389008093880090938B0080937F
:100A00008A0090938D0080938C00259A2D9A2FEF69
:100A100080E792E0215080409040E1F700C0000064
:100A2000269A2E9A2FEF80E792E021508040904046
:100A3000E1F700C00000279A2F9A2FEF80E792E09D
:100A4000215080409040E1F700C0000025982D988B
:100A50002FEF80E792E0215080409040E1F700C006
:100A6000000026982E982FEF80E792E021508040DA
:100A70009040E1F700C0000027982F9856985E98A4
:100A800025982D9826982E9827982F98089589EACA
:100A90008093800089E08093810024982C983F986F
:100AA0008AB18F748AB96E98479A8BB1806B8BB973
:100AB000769A0E94EF040C94B50480E280930001C2
:100AC0008091340181110EC00E94AC0581E08093B9
:100AD00034012FEF83ED90E3215080409040E1F707
:100AE00000C0000080E40E94B205809300018111E3
:100AF0002EC00E94DC0580930001811128C00E9455
:100B0000DC0580930001811122C08FE30E94DC0587
:100B10008093000181111BC00E94D40580E40E94D3
:100B2000B20580930001811112C08CE00E94DC05A7
:100B30008093000181110BC00E94DC0580930001AD
:100B4000811105C08FE30E94DC05809300010E94A3
:100B5000D4058091000108951092B9008AE0809335
:100B6000B800089594EA9093BC009091BC0097FF60
:100B7000FCCF9091B900987F983021F0903111F01E
:100B800081E008958093BB0084E88093BC0080914D
:100B9000BC0087FFFCCF8091B900887F883111F0BD
:100BA000803471F780E0089584E98093BC008091DF
:100BB000BC0084FDFCCF08958093BB0084E8809343
:100BC000BC008091BC0087FFFCCF9091B900987F5A
:100BD00081E0983209F480E0089584E88093BC00B5
:100BE0008091BC0087FFFCCF8091BB00089580916D
:100BF0000001811115C080E40E94B20580930001BC
:100C000081110CC082E10E94DC05809300018111FA
:100C100005C08FEF0E94DC05809300010E94D4057F
:100C200084B1807F84B985B1807F85B98AB1837FA3
:100C30008AB98BB1837F8BB93E98469808950E94FC
:100C40005D05809300010E94F70580B38C7080BB26
:100C500081B3836F81BBE4E4F1E0A6E3B1E01192DC
:100C60001D9281E0E235F807D1F70C944705BF9259
:100C7000CF92DF92EF92FF920F931F93CF93DF9368
:100C800080910001882379F0809135018F5F8093F6
:100C90003501811108C00E945D058093000181111A
:100CA00002C00E94EF0406E311E0C0E0D0E0DD24C2
:100CB000D39482E0C82EEE24E394F12CC73000F5E3
:100CC00080910001811162C080E40E94B20580938E
:100CD0000001811112C082E10E94DC0580930001B5
:100CE00081110BC0C7010C2E01C0880F0A94EAF7CE
:100CF00080950E94DC05809300010E94D40546C0C7
:100D0000CA30A1F028F4C83059F0C93061F005C0EC
:100D1000CC3089F070F0CD3089F0209A289810C03E
:100D2000219A29980DC0229A2A980AC0239A2B98B2
:100D300007C0529A01C0539A5B9802C03E9A4698E7
:100D4000E0EAEA95F1F78FB179995AC092E08170A3
:100D50008D25892B7C9B02C090E001C094E0892BFB
:100D60007D9B02C090E001C098E0892B7E9B02C071
:100D700090E001C090E1892B9FB19095991F992730
:100D8000991F9295990F907E892B0FC08091000139
:100D900081114BC080E40E94B2058093000188233A
:100DA00089F1B12C0E94D4058B2DF8019081981700
:100DB00019F08083C09201010E94F70521960F5F10
:100DC0001F4FCE30D10509F079CF809101018823E2
:100DD00071F1815080930101882339F08FE99FE000
:100DE0000197F1F700C0000022C0A4E4B1E0E6E3FF
:100DF000F1E081918D9391E0E434F907D1F717C0C8
:100E000090E0A5CF83E10E94DC0580930001811171
:100E1000C8CF81E40E94B205809300018111C1CF47
:100E20000E94ED05B82EB094BDCF80E0BECF0E94E9
:100E3000ED0481E0DF91CF911F910F91FF90EF9032
:100E4000DF90CF90BF900895E82FF0E0EC5BFE4F6D
:100E50008081089508958B3B910578F4883A910537
:100E600040F5853A9105D0F48430910508F0B1C081
:100E70008130910509F4ADC06BC0803E910508F446
:100E800067C0883E910508F4A4C09C01205F310929
:100E90002031310508F05CC090650895853A9105D0
:100EA00009F459C0863A910509F458C083E890E4E2
:100EB0000895883A910509F454C0893A910509F4D6
:100EC00053C08A3A910509F452C08B3A910509F44E
:100ED00051C08C3A910509F450C08D3A910509F43E
:100EE0004FC0803B910509F44EC08E3A910509F43C
:100EF0004DC08F3A910509F44CC0813B910509F42E
:100F00004BC0823B910509F44AC0833B910509F42B
:100F100049C0843B910509F448C0853B910509F41B
:100F200047C0863B910509F446C0873B910509F40B
:100F300045C0883B910509F444C0893B910509F4FB
:100F400043C08A3B910509F042C08AE296E40895C5
:100F500080E090E0089581E890E4089582E890E4CC
:100F6000089582EE94E4089589EE94E408958AEE5B
:100F700094E4089585EB94E4089586EB94E4089551
:100F800087EB94E408958CEC94E408958DEC94E45C
:100F9000089583E895E408958AE895E4089582E940
:100FA00095E4089584E995E4089581E296E408952E
:100FB00083E296E4089584E296E4089585E296E457
:100FC000089586E296E4089587E296E4089580E025
:100FD00094E40895089596E0799FF001112494E532
:100FE000899FE00DF11D1124E60FF11DEE0FFF1F8B
:100FF000E851FF4F859194910895880F991F805A69
:101000009040FC01859194910895880F991F80521A
:101010009F4FFC0185919491089526E0729FF00105
:10102000112444E5849FE00DF11D1124E60FF11D0C
:10103000EE0FFF1FE851FF4F25913491C9019A959A
:1010400081159F4110F4C9010895C901905281157D
:10105000904128F4C9019F700E9405080895C901B4
:1010600090538115904120F4C9019927906C0895FF
:10107000211580E5380769F40E94AD159FEF24E340
:101080004CE0915020404040E1F700C000000C943B
:10109000081D213080E5380731F48091CD01816051
:1010A0008093CD010895C90190558115904108F0B4
:1010B00050C0832F99278F70992781309105D9F4DB
:1010C000A9014370552702C0880F991F4A95E2F77E
:1010D0009C68A90164E0440F551F6A95E1F7442715
:1010E0005370842B952B73E0220F331F7A95E1F711
:1010F000207633271DC08230910529F4922F88274E
:10110000816F906A089583309105A9F4A901437015
:10111000552781E090E002C0880F991F4A95E2F7B9
:101120009C6843E0220F331F4A95E1F7207E377019
:10113000822B932B08950497F1F4A901437055274E
:1011400081E090E002C0880F991F4A95E2F79A6803
:10115000E8CFC90190578115904120F4C9019F70D3
:1011600090620895C90190588115904120F4C901F9
:101170009F70906A0895203E3105E0F4203C3105CF
:1011800058F52133310509F470C048F4293231058E
:1011900009F464C02A32310509F46EC074C02933E1
:1011A0003105F1F022383105D9F02533310509F444
:1011B0004EC069C0233E310589F138F4203E310527
:1011C000C1F0223E3105E1F05EC0263E310569F1F5
:1011D000273E3105A9F157C0C9010E94FD070895B6
:1011E0008091E00180FD02C081FF4DC080EE90E063
:1011F0004BC08091E00180FFF9CF89E390E044C0CB
:101200008091E00182FF0EC08091E00184FF03C065
:1012100080E090E039C083EE90E036C08091E0013C
:1012200082FFF2CF82EE90E02FC08091E00183FF39
:101230000BC08091E00184FDEBCF87EE90E024C0ED
:101240008091E00183FFF5CF86EE90E01DC0809194
:10125000E00185FF07C089E290E016C08091E001BF
:1012600085FFF9CF85E390E00FC08091E00186FF14
:1012700007C08AE290E008C08091E00186FFF9CFC4
:1012800081E390E001C0C9010E942B0708950895F1
:101290000C944709809162010895CF93DF9300D0A9
:1012A0001F92CDB7DEB72091E601243019F523E077
:1012B00029839B838A832093E9008FEF9091E80034
:1012C000815095FD06C095ED9A95F1F700008111CA
:1012D000F5CF8091E80085FF0DC040E050E063E06D
:1012E00070E0CE0101960E94B70B8091E8008E77E6
:1012F0008093E8000F900F900F90DF91CF910895A9
:10130000CF93DF9300D01F92CDB7DEB72091E601D7
:10131000243021F522E029839B838A8383E0809314
:10132000E9008FEF9091E800815095FD06C095EDA2
:101330009A95F1F700008111F5CF8091E80085FFC3
:101340000DC040E050E063E070E0CE0101960E94E5
:10135000B70B8091E8008E778093E8000F900F9094
:101360000F90DF91CF9108952091E6012430F1F4A0
:1013700022E02093E9002FEF3091E800215035FD65
:1013800006C035ED3A95F1F700002111F5CF209117
:10139000E80025FF0BC040E050E065E070E00E94EF
:1013A000B70B8091E8008E778093E8000895CF9383
:1013B000DF93EC018091E601843009F046C0909102
:1013C0000C019923D9F090910D019923B9F08093E4
:1013D000E9008FEF9091E800815095FD06C095E1FE
:1013E0009A95F1F700008111F5CF8091E80085FF13
:1013F0002CC040E050E060E170E017C081E08093D5
:10140000E9008FEF9091E800815095FD06C095EDC1
:101410009A95F1F700008111F5CF8091E80085FFE2
:1014200014C040E050E068E070E0CE010E94B70BCD
:101430008091E8008E778093E80080E1FE01A2E5CC
:10144000B1E001900D928A95E1F7DF91CF91089577
:101450008091E501811109C00E94490D0E94A60DED
:101460008091E20084608093E20008951092E5018B
:10147000089508950C942E230E949F1C0E943423EB
:101480000E9443100C94480942E061EC81E00E9404
:10149000C30C42E061EC82E00E94C30C42E061ECCC
:1014A00083E00E94C30C42E161EC84E00C94C30C25
:1014B0008091E801833009F455C030F4813071F037
:1014C000823009F48EC008958A3009F47AC08B30D6
:1014D00009F460C0893009F09CC020C08091E70108
:1014E000813A09F096C08091E800877F8093E800F8
:1014F0008091EB019091EC01892B21F060E080E07C
:1015000090E003C060E182E591E070E00E94000C91
:101510008091E8008B778093E80008958091E7013F
:10152000813209F076C08091EB019091EC01009737
:1015300019F0039709F06DC08091E800877F8093D0
:10154000E8008091E80082FD05C08091E6018111EC
:10155000F8CF5FC08091F100809362018091E80034
:101560008B7753C08091E701813A09F052C0809196
:10157000EB019091EC01892B09F04BC08091E800C0
:10158000877F8093E8008091E80080FFFCCF809106
:101590000C0136C08091E7018132D9F58091EB01D1
:1015A0009091EC01892BA9F58091E800877F8093C9
:1015B000E8000E94F80C8091E90180930C010C94E2
:1015C000AD158091E701813221F58091E800877F98
:1015D0008093E8000E94F80C8091EA0180936301F7
:1015E00008958091E701813AA1F48091E800877F16
:1015F0008093E8008091E80080FFFCCF8091630138
:101600008093F1008091E8008E778093E8000C943D
:10161000F80C089584B7877F84BF88E10FB6F894EB
:1016200080936000109260000FBE90E080E80FB6DB
:10163000F89480936100909361000FBE0E94921015
:101640000E94490D0E94A60D8091E2008460809363
:10165000E20078940E9421100E94941082E091E0B0
:101660000E943E100E941C238091E601853069F49F
:101670000E94621C8091E4018823B1F30E948A1CBD
:10168000882391F30E94A10BEFCF0E949A10ECCF18
:10169000292F332723303105A9F06CF4213031058F
:1016A00009F442C02230310509F043C08DE690E0D4
:1016B00024E037E042C021323105C9F02232310541
:1016C00019F137C099278130910541F08230910599
:1016D00041F0892B71F5E0E0F7E005C0E8EEF6E0B7
:1016E00002C0E0EDF6E0849190E09F0126C06430F6
:1016F00000F5E62FF0E0EE0FFF1FEE5DFE4F2081BC
:10170000318189E090E019C0643098F4E62FF0E070
:10171000DF01AA0FBB1FA65EBE4F2D913C91EA5E72
:10172000FE4F808190E009C082E190E021E737E040
:1017300004C080E090E020E030E0FA0131832083B3
:10174000089580E189BD82E189BD09B400FEFDCF25
:101750008091D8008F7D8093D8008091E0008260D6
:101760008093E0008091E00081FDFCCF0895CF924E
:10177000DF92EF92FF920F931F93CF93DF937C0141
:101780008B01EA010E94190D811131C0209731F0BF
:1017900088819981081B190BE80EF91EC12CD12CE8
:1017A0000115110519F18091E80085FD14C08091A3
:1017B000E8008E778093E800209741F08881998136
:1017C0008C0D9D1D9983888385E011C00E94190DA1
:1017D000882331F30CC0F70181917F018093F100E0
:1017E00001501109FFEFCF1ADF0ADACF80E0DF9155
:1017F000CF911F910F91FF90EF90DF90CF900895C0
:101800002091ED013091EE012617370748F0611560
:10181000710539F42091E8002E772093E80001C08B
:10182000B901FC0120E061157105B9F18091E60173
:10183000882309F440C0853009F43FC08091E80056
:1018400083FD3DC08091E80082FF06C08091E800E2
:1018500082FF26C080E008958091E80080FFE3CFFA
:101860002091F3008091F20090E0922B61157105B8
:1018700051F08830910538F421912093F1006150A6
:1018800071090196F3CF21E0089709F020E08091DB
:10189000E8008E778093E800C6CF2111C7CFD6CF5E
:1018A0008091E601882339F0853039F08091E80095
:1018B00083FFCCCF04C082E0089583E0089581E0E7
:1018C00008952091ED013091EE012617370748F079
:1018D0006115710539F42091E8002E772093E80016
:1018E00001C0B901FC0120E061157105C1F18091D1
:1018F000E601882309F441C0853009F440C0809195
:10190000E80083FD3EC08091E80082FF06C0809120
:10191000E80082FF27C080E008958091E80080FF02
:10192000E3CF2091F3008091F20090E0922B6115BB
:10193000710559F08830910540F424912093F1000D
:101940003196615071090196F2CF21E0089709F0B4
:1019500020E08091E8008E778093E800C5CF2111C8
:10196000C6CFD5CF8091E601882339F0853039F094
:101970008091E80083FFCBCF04C082E0089583E02C
:10198000089581E00895982F973058F59093E900D5
:10199000981739F07091EC002091ED005091F00013
:1019A00003C0242F762F50E021FF19C03091EB00A7
:1019B0003E7F3093EB003091ED003D7F3093ED00A2
:1019C0003091EB0031603093EB007093EC0020938A
:1019D000ED005093F0002091EE0027FF07C09F5FBD
:1019E000D3CF8F708093E90081E0089580E008955F
:1019F0008091E70187FD05C08091E80080FF0EC05F
:101A000012C08091E80082FD05C08091E60181113D
:101A1000F8CF08958091E8008B7708C08091E601A7
:101A20008111EACF08958091E8008E778093E800D5
:101A300008958091E4009091E50045E62091EC0046
:101A400020FF21C02091E80020FD21C02091E60167
:101A5000222389F0253089F02091EB0025FD0FC06D
:101A60002091E4003091E5002817390739F34150FF
:101A700041F0C901E3CF82E0089583E0089581E059
:101A8000089584E008952091E80022FFDFCF80E0F0
:101A900008950E94B70D0E94BF0DE0EEF0E0808136
:101AA00081608083E8EDF0E080818F77808319BCCE
:101AB000A7EDB0E08C918E7F8C9380818F7E8083A8
:101AC0001092E50108950F931F93CF93DF930E9427
:101AD000B70D0E94BF0DC8EDD0E088818F77888355
:101AE00088818068888388818F7D888319BC109263
:101AF000E6011092E2011092E4011092E30100EE7F
:101B000010E0F80180818B7F8083888181608883E9
:101B100042E060E080E00E94C30CE1EEF0E08081F2
:101B20008E7F8083E2EEF0E080818160808380811F
:101B300088608083F80180818E7F808388818061C6
:101B40008883DF91CF911F910F910895E8EDF0E028
:101B500080818F7E8083E7EDF0E0808181608083EB
:101B600084E082BF81E08093E5010C94630DE8ED91
:101B7000F0E080818E7F80831092E20008951092C1
:101B8000DA001092E10008951F920F920FB60F92A3
:101B900011242F933F934F935F936F937F938F9372
:101BA0009F93AF93BF93EF93FF938091E10082FFE8
:101BB0000BC08091E20082FF07C08091E1008B7F23
:101BC0008093E1000E9420108091DA0080FF1FC006
:101BD0008091D80080FF1BC08091DA008E7F8093B7
:101BE000DA008091D90080FF0DC080E189BD82E1DB
:101BF00089BD09B400FEFDCF81E08093E6010E941B
:101C0000280A05C019BC1092E6010E94360A80918C
:101C1000E10080FF19C08091E20080FF15C0809133
:101C2000E2008E7F8093E2008091E20080618093E9
:101C3000E2008091D80080628093D80019BC85E0D2
:101C40008093E6010E943A0A8091E10084FF30C04F
:101C50008091E20084FF2CC080E189BD82E189BDD2
:101C600009B400FEFDCF8091D8008F7D8093D8000D
:101C70008091E1008F7E8093E1008091E2008F7E71
:101C80008093E2008091E20081608093E200809185
:101C9000E201882311F084E007C08091E30087FF10
:101CA00002C083E001C081E08093E6010E943C0A0B
:101CB0008091E10083FF29C08091E20083FF25C06D
:101CC0008091E100877F8093E10082E08093E601CC
:101CD0001092E2018091E1008E7F8093E10080917B
:101CE000E2008E7F8093E2008091E2008061809329
:101CF000E20042E060E080E00E94C30C8091F000CE
:101D000088608093F0000E94390AFF91EF91BF91A3
:101D1000AF919F918F917F916F915F914F913F9183
:101D20002F910F900FBE0F901F9018951F920F923A
:101D30000FB60F9211242F933F934F935F936F939E
:101D40007F938F939F93AF93BF93CF93EF93FF9323
:101D5000C091E900CF708091EC001092E900809171
:101D6000F000877F8093F00078940E94D20E10924A
:101D7000E9008091F00088608093F000C093E90052
:101D8000FF91EF91CF91BF91AF919F918F917F91F3
:101D90006F915F914F913F912F910F900FBE0F90D8
:101DA0001F9018951F93CF93DF93CDB7DEB7AA97F7
:101DB0000FB6F894DEBF0FBECDBFE7EEF1E0809125
:101DC000F100819321E0EF3EF207C9F70E94580A23
:101DD0008091E80083FF1CC12091E7013091E80168
:101DE000832F90E08A30910508F012C1FC01EA5A75
:101DF000FF4F0C94B624203881F0223809F008C136
:101E00008091EB018F708093E9008091EB0085FB5E
:101E1000882780F91092E90006C08091E301909133
:101E2000E401911182609091E800977F9093E8001F
:101E30008093F1001092F100C5C0822F8D7F09F0D0
:101E4000E7C0222319F0223061F0E2C08091E9015D
:101E5000813009F0DDC0333009F080E08093E40187
:101E600028C08091E901811124C02091EB012F70DD
:101E700009F4CEC02093E9008091EB0080FF19C0E7
:101E80008091EB00333011F4806211C08061809347
:101E9000EB0081E090E0022E01C0880F0A94EAF77F
:101EA0008093EA001092EA008091EB0088608093B2
:101EB000EB001092E9008091E800877F86C0211135
:101EC000A7C01091E9011F778091E3008078812BF2
:101ED0008093E3008091E800877F8093E8000E9470
:101EE000F80C8091E80080FFFCCF8091E3008068CF
:101EF0008093E300112311F083E001C082E080931E
:101F0000E60186C02058223008F082C08091E901A5
:101F10009091EA018C3D23E0920779F583E08A8372
:101F20008AE289834FB7F894DE01139620E03EE001
:101F300051E2E32FF0E050935700E49120FF03C0FB
:101F4000E295EF703F5FEF708E2F90E0EA3010F077
:101F5000C79601C0C0968D939D932F5F243149F79A
:101F60004FBF8091E800877F8093E8006AE270E0CD
:101F7000CE0101960E94000C14C0AE014F5F5F4F6E
:101F80006091EB010E94480B009709F441C0209139
:101F9000E800277F2093E800BC0189819A810E9494
:101FA000610C8091E8008B778093E80031C0203885
:101FB00079F58091E800877F8093E8008091E201C5
:101FC0008093F1008091E8008E778093E8000E9472
:101FD000F80C1EC021111CC09091E9019230C0F490
:101FE0008091E800877F8093E8009093E2010E944F
:101FF000F80C8091E201811104C08091E30087FF19
:1020000002C084E001C081E08093E6010E94440A9E
:102010008091E80083FF0AC08091E800877F809369
:10202000E8008091EB0080628093EB00AA960FB6E7
:10203000F894DEBF0FBECDBFDF91CF911F91089501
:102040000895CF938091E6018823B1F08091E90053
:102050008F709091EC0090FF02C090E801C090E07A
:10206000C92FC82B1092E9008091E80083FD0E94DF
:10207000D20ECF70C093E900CF910895909369017B
:10208000809368010895E0916801F09169013097AB
:1020900021F00190F081E02D099480E00895E09115
:1020A0006801F0916901309721F00280F381E02D01
:1020B00009940895E0916801F0916901309721F049
:1020C0000480F581E02D09940895209166013091F6
:1020D00067018217930771F09093670180936601FF
:1020E000E0916801F0916901309721F00680F78155
:1020F000E02D0994089520916401309165018217C3
:10210000930771F09093650180936401E0916801F9
:10211000F0916901309721F00084F185E02D099458
:10212000089508950C9491100E94A51C0E941F060A
:102130000C946B1DCF92DF92EF92FF920F931F933F
:10214000CF93DF93CDB7DEB72B970FB6F894DEBFF2
:102150000FBECDBF0E9437063BE6E32E31E0F32EE3
:1021600000E010E0C02E802F0E942407F701D190DC
:102170007F01D826B1F40F5F1F4F0E30110591F784
:102180008FEF89838A831B820E94AE1C8160782F27
:102190009D838C8349815A816B818D810E943D1181
:1021A00041C09091CD0191FF04C08B870E942A0706
:1021B0008B8520E030E04D2D50E0922FBA01022EA9
:1021C00002C0759567950A94E2F760FF25C02E83DB
:1021D000CF82EE24E394F12C02C0EE0CFF1C9A9502
:1021E000E2F790E08E219F2121E0892B09F420E085
:1021F00028870E94AE1C8160782F9A8789874E813C
:102200005F8168858A850E943D11F801E559FE4F7E
:1022100080818E25808306C02F5F3F4F2630310599
:1022200061F6A9CF0E944F2010916A010E944310CD
:102230001817A1F00E94431080936A012B960FB6E5
:10224000F894DEBF0FBECDBFDF91CF911F910F91EC
:10225000FF90EF90DF90CF900C9448092B960FB62B
:10226000F894DEBF0FBECDBFDF91CF911F910F91CC
:10227000FF90EF90DF90CF900895CF93DF93CDB78D
:10228000DEB72B970FB6F894DEBF0FBECDBF4F83DE
:10229000588769877A878B87DE01119686E0FD0172
:1022A00011928A95E9F785E0FE01379601900D922B
:1022B0008A95E1F749815A816B817C818D819E816C
:1022C0000E9479182B960FB6F894DEBF0FBECDBFD3
:1022D000DF91CF910895CF93C82F882309F4C1C00F
:1022E000823859F40E94431081FDBBC089E30E94EB
:1022F000161B0E94E01B89E30CC0833879F40E940E
:10230000431080FDAEC083E50E94161B0E94E01BB7
:1023100083E50E94561BCF910C94E01B843859F43E
:102320000E94431082FD9DC087E40E94161B0E94FC
:10233000E01B87E4EECF8CEF8C0F813A48F48C2FB2
:102340000E94842281118DC08C2F0E94161BE3CF26
:1023500080E28C0F883048F4C77081E001C0880F9C
:10236000CA95EAF70E94971BD6CF8BE58C0F833076
:1023700078F4C53A29F0C63A31F482E890E005C015
:1023800081E890E002C083E890E0CF910C94651062
:1023900088E58C0F833108F064C0C83A39F1C93A36
:1023A00041F1CA3A49F1CB3A51F1CC3A59F1CD3A1F
:1023B00061F1C03B69F1CE3A71F1CF3A79F1C13B9D
:1023C00081F1C23B89F1C33B91F1C43B99F1C53B1B
:1023D000A1F1C63BA9F1C73BB1F1C83BB9F1C93B7B
:1023E000C1F1CA3BC9F58AE292E038C082EE90E0C2
:1023F00035C089EE90E032C08AEE90E02FC085EBC8
:1024000090E02CC086EB90E029C087EB90E026C0DE
:102410008CEC90E023C08DEC90E020C083E891E04C
:102420001DC08AE891E01AC082E991E017C084E9F2
:1024300091E014C081E292E011C083E292E00EC00C
:1024400084E292E00BC085E292E008C086E292E06E
:1024500005C087E292E002C080E090E0CF910C944A
:102460007B10CF910895882309F44BC0823859F42A
:102470000E94431081FF45C089E30E94161B0E9401
:10248000E01B89E30CC0833871F40E94431080FF85
:1024900038C083E50E94161B0E94E01B83E50E9462
:1024A000561B0C94E01B843859F40E94431082FFA1
:1024B00028C087E40E94161B0E94E01B87E4EFCF30
:1024C0009CEF980F913A58F390E2980F983050F49F
:1024D000877091E001C0990F8A95EAF7892F0E94D1
:1024E0009D1BDFCF9BE5980F933020F480E090E0B8
:1024F0000C946510885A833120F480E090E00C94AD
:102500007B100895882321F00E94971B0C94E01BF8
:102510000895882321F00E949D1B0C94E01B0895D0
:10252000CF92DF92EF92FF920F931F93CF93DF939F
:10253000CDB7DEB728970FB6F894DEBF0FBECDBF7C
:102540008C0185E0F801DE01119601900D928A95CB
:10255000E1F7F80140813181F280258122952F70C9
:1025600083819481892B31F03F3F31F481E04F3FEB
:1025700019F403C081E001C080E080FDCBC2498333
:102580003A8389819A812F830E94D41A9E838887F7
:102590000E94D31A0E94A6192F814E816885FF20C0
:1025A00029F00E94B41B68854E812F81E42FE295AB
:1025B000EF70F0E0E05AFF4F0C94B624842F807F38
:1025C000142F1F70882311F01295107FFF2059F0EF
:1025D000112309F454C2812F68870E94A71B0E940F
:1025E000E01B68854CC2862F0E943312112309F428
:1025F00091C2812F0E94AD1B28960FB6F894DEBFC2
:102600000FBECDBFDF91CF911F910F91FF90EF9043
:10261000DF90CF900C94E01B342F307F842F8F708D
:10262000303211F08295807F662319F0613019F104
:102630002BC0FF20B1F0222309F493C1213009F00F
:1026400090C128960FB6F894DEBF0FBECDBFDF91C4
:10265000CF911F910F91FF90EF90DF90CF900C944E
:10266000C71B222319F0213009F454C28E830E9423
:10267000CA1B8E8189C1FF2021F0223008F04AC296
:1026800070C1211147C280C1FF2021F0222309F42B
:1026900068C1F5C1222309F477C105C2242F26950C
:1026A0002695237030E02115310521F021303105C8
:1026B000C9F030C2FF2021F0862F942F937002C002
:1026C00080E090E028960FB6F894DEBF0FBECDBF35
:1026D000DF91CF911F910F91FF90EF90DF90CF90FE
:1026E0000C946510FF2021F0862F942F937002C068
:1026F00080E090E028960FB6F894DEBF0FBECDBF05
:10270000DF91CF911F910F91FF90EF90DF90CF90CD
:102710000C947B10862FFF2019F00E94571F02C0D7
:102720000E94BF1F28960FB6F894DEBF0FBECDBF24
:10273000DF91CF911F910F91FF90EF90DF90CF909D
:102740000C944420842F837009F076C0F110E2C10C
:10275000262F229526952770220F220F862F8F7005
:10276000C82ED12CE12CF12C022E04C0CC0CDD1C87
:10277000EE1CFF1C0A94D2F764FF10C06FE070E0FB
:1027800080E090E004C0660F771F881F991F2A958C
:10279000D2F7609570958095909503C060E070E0E9
:1027A000CB01242F269526952370422F50E04230EE
:1027B0005105D1F04330510559F16C297D298E29FD
:1027C0009F294130510541F128960FB6F894DEBF9C
:1027D0000FBECDBFDF91CF911F910F91FF90EF9072
:1027E000DF90CF900C94CB196C297D298E299F29DD
:1027F00028960FB6F894DEBF0FBECDBFDF91CF9104
:102800001F910F91FF90EF90DF90CF900C94E519FE
:102810000E94CB19C701B60128960FB6F894DEBF07
:102820000FBECDBFDF91CF911F910F91FF90EF9021
:10283000DF90CF900C94B119FF2019F0842F817094
:1028400001C08695882309F465C1262F2295269517
:102850002770220F220F862F8F70C82ED12CE12CCB
:10286000F12C022E04C0CC0CDD1CEE1CFF1C0A94C3
:10287000D2F764FF10C06FE070E080E090E004C029
:10288000660F771F881F991F2A95D2F7609570955C
:102890008095909503C060E070E0CB01242F2695D1
:1028A00026952370422F50E042305105D1F043303D
:1028B000510559F16C297D298E299F2941305105F7
:1028C00041F128960FB6F894DEBF0FBECDBFDF9161
:1028D000CF911F910F91FF90EF90DF90CF900C94CC
:1028E0009F1A6C297D298E299F2928960FB6F89466
:1028F000DEBF0FBECDBFDF91CF911F910F91FF9033
:10290000EF90DF90CF900C94B91A0E949F1AC701E4
:10291000B60128960FB6F894DEBF0FBECDBFDF918B
:10292000CF911F910F91FF90EF90DF90CF900C947B
:10293000851A603FC9F118F4603E50F49BC0623FB5
:1029400009F460C008F44AC0633F09F46FC092C044
:10295000162F1F70842F8F71FF2099F00E941E1A6E
:10296000812F28960FB6F894DEBF0FBECDBFDF9142
:10297000CF911F910F91FF90EF90DF90CF900C942B
:1029800082120E943F1A812F28960FB6F894DEBF5C
:102990000FBECDBFDF91CF911F910F91FF90EF90B0
:1029A000DF90CF900C948912FF20A1F02111B2C0CA
:1029B000842F8F7128960FB6F894DEBF0FBECDBF5F
:1029C000DF91CF911F910F91FF90EF90DF90CF900B
:1029D0000C94641A223008F09DC0EACFFF20A1F0C9
:1029E000842F8F7128960FB6F894DEBF0FBECDBF2F
:1029F000DF91CF911F910F91FF90EF90DF90CF90DB
:102A00000C941E1AFF2061F3842F8F7128960FB645
:102A1000F894DEBF0FBECDBFDF91CF911F910F9114
:102A2000FF90EF90DF90CF900C943F1AFF2091F031
:102A3000842F8F7128960FB6F894DEBF0FBECDBFDE
:102A4000DF91CF911F910F91FF90EF90DF90CF908A
:102A50000C94091A28960FB6F894DEBF0FBECDBFAE
:102A6000DF91CF911F910F91FF90EF90DF90CF906A
:102A70000C94FF19FF20A1F0222309F4B1CF862F77
:102A800028960FB6F894DEBF0FBECDBFDF91CF9171
:102A90001F910F91FF90EF90DF90CF900C946B11EE
:102AA000222309F4B1CF862F28960FB6F894DEBF03
:102AB0000FBECDBFDF91CF911F910F91FF90EF908F
:102AC000DF90CF900C9433124F70C8010E94A50480
:102AD00028960FB6F894DEBF0FBECDBFDF91CF9121
:102AE0001F910F91FF90EF90DF90CF900C942619DB
:102AF0004F70C80128960FB6F894DEBF0FBECDBF49
:102B0000DF91CF911F910F91FF90EF90DF90CF90C9
:102B10000C94EA0728960FB6F894DEBF0FBECDBF1F
:102B2000DF91CF911F910F91FF90EF90DF90CF90A9
:102B300008950E94B41B0E94C41B0E94891B0E941E
:102B4000E01B0E94F0200E94442080E090E00E9460
:102B5000651080E090E00C947B100E94A41B0C9404
:102B600099150E94D41A292F22952F7030E02C300D
:102B700031054CF42A3031056CF4225031092230F1
:102B8000310590F407C02C30310551F02F3031055C
:102B900039F00AC0803E10F0803F31F481E00895A2
:102BA00093FB882780F9089580E00895CF93DF9301
:102BB00000D000D01F92CDB7DEB70F900F900F90CE
:102BC0000F900F90DF91CF910895CF93DF9300D0B6
:102BD00000D000D0CDB7DEB726960FB6F894DEBF92
:102BE0000FBECDBFDF91CF9108951F93CF93DF9399
:102BF000C091790116E080917A01C81799F0D0E070
:102C00001C9FF0011D9FF00D1124E558FE4F4081DF
:102C1000518162817381848195810E94E51521969D
:102C2000C770E9CFDF91CF911F9108954091AB011B
:102C30005091AC016091AD017091AE018091AF01F6
:102C40009091B0010C94E515CF938091B0018295DD
:102C50008F7009F05FC08091AD01882309F45AC0DC
:102C600020917901A0917A016091AB017091AC0142
:102C70008091AE019091AF0131E06F3F09F030E0FB
:102C8000B32FC6E02A1709F445C0009721F07F3F13
:102C900021F44B2F03C041E001C040E030E040FD93
:102CA00035C0C29FF001C39FF00D1124E558FE4FBF
:102CB000418174132BC04081641328C042814111AB
:102CC00025C0438154814817590710F441505109D8
:102CD000481B590B483C5105C8F48091B0018F70D6
:102CE00080618093B00186E0829FF001839FF00DA8
:102CF0001124E058FE4F80818F70806180838BEAC1
:102D000091E00E949012CF910C94F5152F5F3F4FE8
:102D10002770B8CFCF910895CF92DF92EF92FF92B4
:102D20000F931F93CF93DF93CDB7DEB762970FB6A4
:102D3000F894DEBF0FBECDBF8C0185E0F801DE0147
:102D40001D9601900D928A95E1F7D8014C9111964C
:102D50005C91119712966C9112971396ED90FC90DE
:102D600014977091AB01E091AC012091AE013091CC
:102D7000AF012115310531F0EF3F31F481E07F3FA4
:102D800019F403C081E001C080E0B82FB170CB2EF0
:102D900080FD6CC1D090AD01DD2009F4F5C0F0914B
:102DA000B001E216F30638F0C701821B930B883C92
:102DB000910548F09BC0209530952E0D3F1D283C75
:102DC000310508F093C08F2F807F09F052C0E513C2
:102DD00014C0741312C0D62E61110FC0FF70F061C1
:102DE000F093B0010E9416168BEA91E00E949012B7
:102DF0008091B001F80185836CC1EF2831F05F3F0D
:102E000031F481E04F3F19F403C081E001C080E05C
:102E100080FD03C081E0862701C080E0F82FF170BB
:102E2000FF2E80FF1CC08091790120917A0136E04D
:102E3000821709F428C190E0389FF001399FF00D06
:102E40001124E558FE4F7181571306C07081471356
:102E500003C07281671303C001968770E9CFD62E35
:102E6000662309F436C18091B00181608093B0017E
:102E700053C0E51308C0741306C0611104C0D80123
:102E80001596FC93AEC04D875E878D859E856A8BB7
:102E90000E94B1156A89882329F1D62E662311F183
:102EA0002091B001822F82958F7090E002970CF4F0
:102EB00060C08091AB019091AC0198878F83198697
:102EC000FB86EA862C87CE01079651C0E51731F1C3
:102ED0004D875E878D859E856A8B0E94B1156A89B4
:102EE00081112EC0C8010E949012A4C08F2F807F34
:102EF00069F77E2DF98AE88A89890E94D6158BEABE
:102F000091E00E949012EBEAF1E086E0DF011D9271
:102F10008A95E9F70E941616D12CDBC07413D8CF1E
:102F20006111D6CFD8011596FC93C8010E9490126A
:102F3000EBEAF1E086E0DF011D928A95E9F7C9C06E
:102F4000D62E662379F22091B001822F82958F7060
:102F500090E0029774F08091AB019091AC019A835C
:102F600089831B82FD82EC822E83CE0101960E9412
:102F7000901286E0F801ABEAB1E001900D928A95DB
:102F8000E1F70E9424166FC0E216F30628F0C7018D
:102F9000821B930B9C0104C0209530952E0D3F1D84
:102FA000283C310508F052C0D62E662309F49ACF8A
:102FB000E5132CC074132AC08091B00180FD1DC0A0
:102FC000982F92959F70C9F0D80115968C931597FC
:102FD0009F3039F09F5F9295907F8F70892B159667
:102FE0008C93C8010E94901286E0F801ABEAB1E030
:102FF00001900D928A95E1F736C086E0F801ABEAC0
:10300000B1E001900D928A95E1F763C04D875E872C
:103010008D859E850E94B115882379F086E0F801A0
:10302000ABEAB1E001900D928A95E1F70E94241677
:103030000E941616DD24D3944CC08091B0018160AB
:103040008093B001C8010E94901243C07E2DF98A7E
:10305000E88A89890E94D615EBEAF1E086E0DF0173
:103060001D928A95E9F70E94161633C0662309F46B
:1030700039CF4D875E878D859E850E94B115882347
:1030800009F430CFCBCF4D875E878D859E850E941A
:10309000D41A292F22952F7030E0223031052CF4DC
:1030A0009F7041F0811106C00CC0243031052CF412
:1030B0009F7049F4805E883020F0C8010E94901211
:1030C000CF2CDC2C06C0D80115969C91907F91F7EF
:1030D000F8CF8D2D62960FB6F894DEBF0FBECDBF30
:1030E000DF91CF911F910F91FF90EF90DF90CF90E4
:1030F00008951F93CF93DF93CDB7DEB72C970FB60C
:10310000F894DEBF0FBECDBF4F83588769877A879B
:103110008B879C87CE0107960E948C168823C1F06E
:103120002F8138858A859B85892B31F03F3F11F0AF
:1031300080E003C02F3FE1F781E0811147C04F815C
:10314000588569857A858B859C850E94E5153EC0EA
:1031500086E0FE013796DE01119601900D928A9568
:10316000E1F7FF81E8854A855B854115510531F01E
:10317000EF3F31F481E0FF3F19F403C081E001C06B
:1031800080E080FD23C020917A0130E0C9010196E2
:10319000877099276091790170E086179707F1F1A0
:1031A000F983EA835D834C8396E0929FD001939FDD
:1031B000B00D1124A558BE4FFE01319601900D921D
:1031C0009A95E1F780937A010E94F51516E08091B7
:1031D000790190917A01891779F1189FC001112422
:1031E00085589E4F0E948C16882331F1E091790119
:1031F0001E9FF0011124E558FE4F408151816281EC
:103200007381848195810E94E5158091790190E018
:1032100001968770992780937901D9CF0E94AD15C7
:1032200010927A0110927901EBEAF1E086E0DF0179
:103230001D928A95E9F7CACF2C960FB6F894DEBF97
:103240000FBECDBFDF91CF911F910895EF92FF92F6
:103250000F931F93CF93DF93FC01009709F46FC086
:10326000F12CEE24E394EF0121968491843740F40D
:10327000843008F055C0813081F0823021F15FC088
:10328000853709F447C0C0F19CE7980F903708F0E4
:1032900056C08F770E94331245C08F010E5F1F4FBB
:1032A000FE01849190E2980F983050F48770FE2DC3
:1032B00001C0FF0F8A95EAF78F2F0E94B71B15C038
:1032C0000E946B1114C08F010E5F1F4FFE0184918D
:1032D00090E2980F983068F48770FE2D01C0FF0FC0
:1032E0008A95EAF78F2F0E94BD1B0E94E01BE80120
:1032F00019C00E943312FBCFCF010296FE01C49188
:10330000CC2361F0EFE9FFE03197F1F700C0000056
:10331000C150F6CFCF010296FE01F490EC0102C03D
:103320000E946B118F2D882341F0EFE9FFE0319768
:10333000F1F700C000008150F6CFFE0194CFDF917D
:10334000CF911F910F91FF90EF9008950895609392
:10335000B5017093B6018093B7019093B8010C94B6
:1033600099150F931F930091B5011091B60120910B
:10337000B7013091B801062B172B282B392B00935E
:10338000B5011093B6012093B7013093B8011F9196
:103390000F910C9499150F931F930091B501109103
:1033A000B6012091B7013091B801062317232823D5
:1033B00039230093B5011093B6012093B7013093E0
:1033C000B8011F910F910C9499150F931F930091C1
:1033D000B5011091B6012091B7013091B8010627CF
:1033E0001727282739270093B5011093B60120939A
:1033F000B7013093B8011F910F910C949915109259
:10340000B1011092B2011092B3011092B4010C9468
:10341000991541E050E060E070E004C0440F551F92
:10342000661F771F8A95D2F74093B1015093B2017E
:103430006093B3017093B4010C94991541E050E08E
:1034400060E070E004C0440F551F661F771F8A9527
:10345000D2F78091B1019091B201A091B301B091E6
:10346000B401842B952BA62BB72B8093B10190939D
:10347000B201A093B301B093B4010C94991541E04B
:1034800050E060E070E004C0440F551F661F771FD6
:103490008A95D2F740955095609570958091B101CD
:1034A0009091B201A091B301B091B401842395230E
:1034B000A623B7238093B1019093B201A093B301E7
:1034C000B093B4010C94991541E050E060E070E0D5
:1034D00004C0440F551F661F771F8A95D2F780914D
:1034E000B1019091B201A091B301B091B4018427D0
:1034F0009527A627B7278093B1019093B201A09397
:10350000B301B093B4010C9499150F931F930091DC
:10351000B1011091B2012091B3013091B401062B99
:10352000172B282B392B0093B1011093B201209354
:10353000B3013093B4011F910F910C9499150F931F
:103540001F930091B1011091B2012091B30130910C
:10355000B40106231723282339230093B1011093C4
:10356000B2012093B3013093B4011F910F910C94D9
:1035700099150F931F930091B1011091B201209101
:10358000B3013091B4010627172728273927009364
:10359000B1011093B2012093B3013093B4011F9194
:1035A0000F910C9499150895CF92DF92EF92FF92AC
:1035B0000F931F93CF93DF93EC01C090B501D09090
:1035C000B601E090B701F090B8018091B1019091FF
:1035D000B201A091B301B091B401C82AD92AEA2A54
:1035E000FB2A0FE110E0B701A601002E04C076957A
:1035F0006795579547950A94D2F740FF07C0BE01DB
:10360000802F0E940D088130910539F40150110975
:1036100050F7BE0180E00E940D08DF91CF911F910D
:103620000F91FF90EF90DF90CF90089590910C0153
:103630009923D9F090910D019923B9F0982F96957F
:10364000969596959F3088F5E0910E01F0910F01C7
:10365000E90FF11D877021E030E001C0220F8A954B
:10366000EAF78181822B8183089540910E01509168
:103670000F0120E030E09FEFFA01E20FF31F6281BB
:10368000681799F09F3F19F4611101C0922F2F5FC5
:103690003F4F2E30310581F79F3F39F0FA01E90F96
:1036A000F11D97FDFA9582830895089590910C017C
:1036B0009923E1F090910D019923C1F0982F9695EF
:1036C000969596959F3020F5E0910E01F0910F01AF
:1036D000E90FF11D877021E030E001C0220F8A95CB
:1036E000EAF72095818128232183089540910E01D6
:1036F00050910F0120E030E0FA01E20FF31F9281B8
:10370000981301C012822F5F3F4F2E303105A1F771
:10371000089581E090E0E0910E01F0910F01E80F33
:10372000F91F1082019680319105A9F708959091B3
:10373000CC01982B9093CC01089580959091CC0169
:1037400098239093CC0108951092CC010895909104
:10375000CB01982B9093CB01089580959091CB014C
:1037600098239093CB0108951092CB0108959091E6
:10377000CA01982B9093CA01089580959091CA012F
:1037800098239093CA0108951092CA0108958093D6
:10379000B90108951092B901089540910E01509118
:1037A0000F0120E030E080E0FA01E20FF31F918189
:1037B00091118F5F2F5F3F4F2F303105A9F708958B
:1037C000E0910E01F0910F018091CC018083E09196
:1037D0000E01F0910F0180819091CB01892B8083A4
:1037E000E0910E01F0910F0180819091CA01892B27
:1037F00080839091B901992361F0E0910E01F091DD
:103800000F018081892B80830E94CD1B8111109232
:10381000B90180910E0190910F010C944F10CF923D
:10382000DF92EF92FF920F931F936C01EE24FF241F
:10383000C114D104E104F10421F46B017C0180E0A6
:1038400001C080E133272F2D1E2D0D2D01151105EF
:103850002105310519F0885F68017901970186011A
:10386000A4E03695279517950795AA95D1F70115E8
:1038700011052105310519F08C5F68017901970167
:103880008601F2E03695279517950795FA95D1F7B9
:10389000011511052105310519F08E5F68017901C7
:1038A000B701A6017695679557954795452B462B09
:1038B000472B09F08F5F1F910F91FF90EF90DF90E2
:1038C000CF9008958091E601843009F11092CE01E5
:1038D00020E488E190E00FB6F894A895809360000A
:1038E0000FBE2093600083B7817F846083BF83B75E
:1038F000816083BF7894889583B78E7F83BF88E18A
:103900000FB6F89480936000109260000FBE089587
:1039100008950895CF930E94881C0E9437060E9444
:10392000891CC0E08C2F0E942407811105C0CF5F45
:10393000CE30C1F780E001C081E0CF9108950E94B0
:10394000AD150E9443100C94480982E084BD93E0B9
:1039500095BD9AEF97BD80936E0008952FB7F894A8
:103960008091CF019091D001A091D101B091D2016D
:103970002FBF0895CF92DF92EF92FF920F931F9384
:103980002FB7F8944091CF015091D0016091D101AF
:103990007091D2012FBF6A017B01EE24FF248C01BC
:1039A00020E030E0C016D106E206F30610F44150E4
:1039B0005109481B590BCA011F910F91FF90EF90BD
:1039C000DF90CF9008951F920F920FB60F9211249F
:1039D0008F939F93AF93BF938091CF019091D0012C
:1039E000A091D101B091D2010196A11DB11D80938A
:1039F000CF019093D001A093D101B093D201BF9198
:103A0000AF919F918F910F900FBE0F901F901895BF
:103A10000E94490DF8942FEF87EA91E621508040EB
:103A20009040E1F700C0000087E090EBDC0180935C
:103A3000EF019093F001A093F101B093F2012CE01B
:103A400088E190E00FB6F894A895809360000FBECF
:103A500020936000FFCFEF92FF920F931F93CF93BD
:103A6000DF93E82EF12C8F2D0E942407C0E0D0E0D8
:103A7000082F10E098010C2E02C0359527950A9466
:103A8000E2F720FD05C02196C630D10599F709C09F
:103A90006C2F7F2D80E00E94EB07E812F4CF81E0CD
:103AA00005C0F3948EE0F812DECF80E0DF91CF9175
:103AB0001F910F91FF90EF900895CF93C82F8CE244
:103AC0000E942B1D882321F08C2FCF910C942B1D4D
:103AD00080E0CF910895CF930E94B01E811102C063
:103AE0000E94961EC5E6C15049F00E9437068FE33A
:103AF0009CE90197F1F700C00000F5CF89E20E9430
:103B00005D1D811111C18AE20E945D1D81110E941B
:103B1000961E85E00E945D1D81110E94081D0E9475
:103B2000BB1E8093CD0187E00E945D1D882399F123
:103B30008BE10E945D1D882351F09091CD0191FB96
:103B4000882780F921E0822780FB91F922C08EE04E
:103B50000E945D1D882351F09091CD0192FB882732
:103B600080F921E0822780FB92F913C080E10E9456
:103B70005D1D9091CD01882341F093FB882780F94A
:103B800021E0822780FB93F904C0892F809580FB78
:103B900090F99093CD018091CD010E94BF1E0E94AB
:103BA000CD1E8093E00180EE0E945D1D882341F0D0
:103BB0008091E001982F909590FB80F98093E0012F
:103BC00089E30E945D1D882359F09091E00191FBEB
:103BD000882780F921E0822780FB91F99093E0010A
:103BE00082EE0E945D1D882359F09091E00192FBC6
:103BF000882780F921E0822780FB92F99093E001E9
:103C000086EE0E945D1D882359F09091E00193FBA0
:103C1000882780F921E0822780FB93F99093E001C7
:103C200083EE0E945D1D882359F09091E00194FB82
:103C3000882780F921E0822780FB94F99093E001A6
:103C400085E30E945D1D882359F09091E00195FB6A
:103C5000882780F921E0822780FB95F99093E00185
:103C600081E30E945D1D882359F09091E00196FB4D
:103C7000882780F921E0822780FB96F99093E00164
:103C800081E10E945D1D882359F09091E00197FB2E
:103C9000882780F921E0822780FB97F99093E00143
:103CA0008091E0010E94D11E8091E00187FB88276E
:103CB00080F980930D0187E20E945D1DC82F8EE17F
:103CC0000E945D1D8111C2608FE10E945D1D811106
:103CD000C46080E20E945D1D8111C86081E20E9483
:103CE0005D1D8111C06182E20E945D1D8111C06273
:103CF00083E20E945D1D8111C06484E20E945D1D0B
:103D0000882311F0C06802C0CC2329F08C2F0E94B8
:103D1000C81E6C2F03C00E94C41E682F70E080E094
:103D200090E0CF910C94A719CF9108956DEE7EEF9E
:103D300080E090E00E94EC2460E082E090E00E944D
:103D4000DE2460E083E090E00E94DE2460E084E016
:103D500090E00E94DE2460E085E090E00C94DE2498
:103D600080E090E00E94D82421E08D3E9E4F09F033
:103D700020E0822F089582E090E00C94D024682FF8
:103D800082E090E00C94DE2483E090E00C94D02458
:103D9000682F83E090E00C94DE2484E090E00C94A3
:103DA000D024682F84E090E00C94DE248091D5012B
:103DB00080FF0BC06091130185E0689FB001112462
:103DC00075956795759567952AC081FF09C06091C3
:103DD000130185E0689FB0011124759567951FC098
:103DE00082FF07C06091130185E0689FB001112434
:103DF00016C04091D6014423C9F0609112014617C4
:103E000088F72091130185E0289F90011124429F9B
:103E1000C001439F900D112470E00E94A2246038DD
:103E2000710540F46115710539F002C065E070E07C
:103E3000862F08958FE7089581E008958091D50138
:103E400080FF08C06091110170E0759567957595C8
:103E5000679521C081FF06C06091110170E07595E2
:103E6000679519C082FF04C06091110170E010C015
:103E70008091D6018823C1F0609110018617A0F7C8
:103E800090911101989FC001112470E00E94A2241A
:103E90006038710528F46115710521F0862F0895A9
:103EA0008FE7089581E0089561E070E0F4CF803FEE
:103EB00021F40E94D61E819504C0813F29F40E94FE
:103EC000D61E8093D9010895823F21F40E94D61E08
:103ED000819504C0833F29F40E94D61E8093D801A7
:103EE0000895893F19F40E941E1F05C08A3F31F4CE
:103EF0000E941E1F81958093DA0108958B3F21F463
:103F00000E941E1F819504C08C3F29F40E941E1F31
:103F10008093DB010895843F21F48091D701816073
:103F200017C0853F21F48091D701826011C0863F80
:103F300021F48091D70184600BC0873F21F48091E8
:103F4000D701886005C0883F31F48091D701806136
:103F50008093D70108958D3F21F48091D501816030
:103F60000BC08E3F21F48091D501826005C08F3F48
:103F700029F48091D50184608093D5010895803F14
:103F800039F48091D90187FF6CC01092D90169C0C2
:103F9000813F29F48091D9011816BCF362C0909139
:103FA000D801823F29F497FF5CC01092D80159C014
:103FB000833F19F41916CCF354C0893F41F4809122
:103FC000DA0118160CF04DC01092DA014AC08A3F8F
:103FD00029F48091DA0187FF44C0F6CF8B3F39F492
:103FE0008091DB0187FF3DC01092DB013AC08C3F1E
:103FF00029F48091DB011816BCF333C0843F21F40F
:104000008091D7018E7F17C0853F21F48091D70121
:104010008D7F11C0863F21F48091D7018B7F0BC02B
:10402000873F21F48091D701877F05C0883F31F415
:104030008091D7018F7E8093D70113C08D3F21F4EB
:104040008091D5018E7F0BC08E3F21F48091D501E8
:104050008D7F05C08F3F29F48091D5018B7F8093A0
:10406000D5018091D80181110EC08091D9018111B3
:104070000AC08091DA01811106C08091DB018111B3
:1040800002C01092D601089587ED91E00E945A1067
:104090000E94AE1C9093D4018093D30108951F9386
:1040A000CF93DF938091D3019091D4010E94BA1CE9
:1040B0004091D601442321F02091140130E006C044
:1040C000209115015AE0259F900111248217930732
:1040D00008F482C08091D8011091D901D091DA0101
:1040E000C091DB01811107C0111105C0D11103C0BE
:1040F000CC2309F471C04F3F19F04F5F4093D601B4
:10410000181624F40E94D61E8093D8018091D801FD
:1041100087FF05C00E94D61E81958093D801111695
:1041200024F40E94D61E8093D9018091D90187FF83
:1041300005C00E94D61E81958093D9016091D80157
:10414000662339F11091D901112319F1772767FD01
:104150007095872F972F0E94B32323E333E343E324
:104160005FE30E9417240E9480236093D801612F8F
:10417000772767FD7095872F972F0E94B32323E33E
:1041800033E343E35FE30E9417240E94802360939C
:10419000D9011D1624F40E941E1F8093DA0180911C
:1041A000DA0187FF05C00E941E1F81958093DA0106
:1041B0001C1624F40E941E1F8093DB018091DB01FA
:1041C00087FF05C00E941E1F81958093DB01DF9150
:1041D000CF911F910C944420DF91CF911F910895AE
:1041E000E7EDF1E085E0DF011D928A95E9F7109295
:1041F000D6011092D5010895833081F128F48130E1
:1042000059F08230D1F00895853009F449C0B8F1F1
:10421000863009F456C0089520911501862F90E04C
:10422000820F911D8F3F910520F4620F609315015D
:1042300008958FEF80931501089520911401862F22
:1042400090E0820F911D8F3F910520F4620F6093E3
:10425000140108958FEF80931401089520911301A4
:10426000862F90E0820F911D8F3F910520F4620F01
:104270006093130108958FEF8093130108952091A7
:104280001201862F90E0820F911D8F3F910520F43F
:10429000620F6093120108958FEF809312010895C9
:1042A00020911101862F90E0820F911D8F3F910583
:1042B00020F4620F6093110108958FEF8093110134
:1042C000089520911001862F90E0820F911D8F3F5D
:1042D000910520F4620F6093100108958FEF809391
:1042E00010010895833011F128F4813049F08230B3
:1042F00091F00895853081F120F18630C1F1089563
:1043000080911501681720F4861B8093150108958C
:1043100010921501089580911401681720F4861BEE
:10432000809314010895109214010895809113014F
:10433000681720F4861B80931301089510921301CF
:10434000089580911201681720F4861B8093120152
:10435000089510921201089580911101681720F4B8
:10436000861B809311010895109211010895809188
:104370001001681720F4861B809310010895109295
:10438000100108958D3109F442C020F58E3009F4F2
:1043900079C070F4873009F45EC020F4863009F4E7
:1043A00042C033C08830D1F18B3009F4A7C02DC092
:1043B000863109F4A3C038F4803109F46DC081312D
:1043C00009F47BC022C0893109F498C08B3109F40B
:1043D0004FC01BC0853309F479C048F4873209F413
:1043E00075C008F478C0893209F470C00EC08334F7
:1043F00038F48A3308F071C0883309F47FC005C0EF
:10440000833409F463C08834C1F080E008950E94C9
:104410003A230E9443100E94480970C00E94BB1EAC
:104420000E94CD1E6BC08091CD01817F8E7F8093D5
:10443000CD0181E08093DD0108950E94AD152FEF3D
:1044400083ED90E3215080409040E1F700C00000F0
:104450000E94081D53C09091CD01892F817090FF5B
:1044600003C0917F9E7F26C091609093CD0146C08E
:104470009091CD0191FB882780F921E0822780FB74
:1044800091F913C09091CD0192FB882780F921E02A
:10449000822780FB92F909C09091CD0193FB882778
:1044A00080F921E0822780FB93F99093CD01882346
:1044B00029F191609093CD0108950E94AD158091EE
:1044C0000D0191E0892780930D0118C061E070E033
:1044D00080E090E00FC023EE01C027EC280F61E0E0
:1044E00070E080E090E004C0660F771F881F991F7E
:1044F0002A95D2F70E94A7190E94AD1581E0089570
:1045000080E0089580E00895CF93C82F8091DD0169
:10451000813079F018F08230D1F184C0A0910E0181
:10452000B0910F018C91813169F0823209F07CC029
:1045300009C0A0910E01B0910F018C91813111F051
:10454000823249F48C2F0E94802281111DC08C2F51
:104550000E94C2211AC08C2F0E948222811114C095
:10456000C43179F048F4CB3079F0C03109F060C043
:1045700082E08093DD0108C0C93219F0C83321F010
:1045800057C01092DD0154C081E0817053C0C93220
:1045900089F118F5C43171F1A8F4C73009F046C0AB
:1045A0008AE08093150194E19093140193E0909335
:1045B00013018093120188E08093110188E28093B7
:1045C000100134C0CE51C63088F5EC2FF0E0E65D26
:1045D000FE4F80818093DC0129C0CE34E9F020F4C5
:1045E000CB3421F56AE013C0C13579F0C235F1F45E
:1045F00061E00DC08091DC01882319F01092DC018C
:1046000015C081E08093DD0115C061E006C0809196
:10461000DC010E94FC200AC06AE08091DC010E945B
:10462000722104C01092DD0180E004C081E002C06C
:1046300080E0ABCFCF910895E1E8F0E08081886021
:1046400080838081816080838FB7F89493E090931A
:10465000890090ED909388008FBF0895EFE6F0E019
:104660008081826080830895EFE6F0E080818D7F15
:1046700080830895EFE6F0E0808192E089278083CF
:1046800008951F920F920FB60F9211242F933F930C
:104690004F935F936F937F938F939F93AF93BF934A
:1046A000EF93FF938091DE019091DF01019690934B
:1046B000DF018093DE01811103C082E00E9448097E
:1046C000E091DF01E695E695F0E0E258F74FE491DE
:1046D0008091DE018E1303C080E00E944809FF91A3
:1046E000EF91BF91AF919F918F917F916F915F916A
:1046F0004F913F912F910F900FBE0F901F901895E3
:1047000004D06894B1118DC0089570D088F09F577F
:1047100090F0B92F9927B751A0F0D1F0660F771F0D
:10472000881F991F1AF0BA95C9F712C0B13081F0ED
:1047300077D0B1E0089574C0672F782F8827B85FCD
:1047400039F0B93FCCF3869577956795B395D9F74E
:104750003EF490958095709561957F4F8F4F9F4F58
:104760000895E89409C097FB3EF490958095709564
:1047700061957F4F8F4F9F4F9923A9F0F92F96E9AD
:10478000BB279395F695879577956795B795F11122
:10479000F8CFFAF4BB0F11F460FF1BC06F5F7F4FBF
:1047A0008F4F9F4F16C0882311F096E911C07723D1
:1047B00021F09EE8872F762F05C0662371F096E8DA
:1047C000862F70E060E02AF09A95660F771F881FA9
:1047D000DAF7880F9695879597F9089557FD9058C1
:1047E000440F551F59F05F3F71F04795880F97FBB5
:1047F000991F61F09F3F79F087950895121613066F
:104800001406551FF2CF4695F1DF08C0161617069D
:104810001806991FF1CF86957105610508940895D2
:10482000E894BB2766277727CB0197F908950BD02B
:1048300078C069D028F06ED018F0952309F05AC0DE
:104840005FC01124EECFCADFA0F3959FD1F3950F7F
:1048500050E0551F629FF001729FBB27F00DB11D04
:10486000639FAA27F00DB11DAA1F649F6627B00D94
:10487000A11D661F829F2227B00DA11D621F739F7D
:10488000B00DA11D621F839FA00D611D221F749F8B
:104890003327A00D611D231F849F600D211D822FD2
:1048A000762F6A2F11249F5750408AF0E1F0882319
:1048B0004AF0EE0FFF1FBB1F661F771F881F915026
:1048C0005040A9F79E3F510570F014C0AACF5F3F3A
:1048D000ECF3983EDCF3869577956795B795F79559
:1048E000E7959F5FC1F7FE2B880F911D96958795E1
:1048F00097F9089597F99F6780E870E060E0089560
:104900009FEF80EC089500240A94161617061806E7
:104910000906089500240A941216130614060506C3
:104920000895092E0394000C11F4882352F0BB0F54
:1049300040F4BF2B11F460FF04C06F5F7F4F8F4FB7
:104940009F4F089597FB072E16F4009407D077FD2C
:1049500009D00E94BC2407FC05D03EF490958195B7
:104960009F4F0895709561957F4F0895EE0FFF1F3B
:104970000590F491E02D0994AA1BBB1B51E107C0DF
:10498000AA1FBB1FA617B70710F0A61BB70B881FDF
:10499000991F5A95A9F780959095BC01CD0108956E
:1049A000F999FECF92BD81BDF89A992780B50895F7
:1049B000A8E1B0E042E050E00C94F324262FF999EE
:1049C000FECF1FBA92BD81BD20BD0FB6F894FA9AF2
:1049D000F99A0FBE019608950E94DE24272F0C94A9
:1049E000DF24DC01CB01FC01F999FECF06C0F2BD4A
:1049F000E1BDF89A319600B40D9241505040B8F79D
:064A00000895F894FFCFB9
:104A060020024A09D709B40980094D090101BA01F2
:104A160028080A03140A3F4D36393F08F207BC0737
:104A2600830716072F0748076107010203040506D7
:044A36000708090064
:00000001FF
